:020000040800F2
:1000000048050020C9000008C5120008AF1100080B
:1000100000000000000000000000000000000000E0
:10002000000000000000000000000000C9120008ED
:100030000000000000000000C7120008CB120008FA
:10004000DB00000800000000DB000008DB00000807
:10005000DB000008DB000008DB000008DB00000814
:1000600000000000DB000008DB000008DB000008E7
:10007000DB000008DB000008DB00000800000000D7
:10008000DB0000080000000000000000DB000008AA
:1000900000000000DB000008DB000008DB000008B7
:1000A00000000000DB000008000000000D1A00083E
:1000B0000448854600F090F800480047B11A00084F
:1000C000C046C04648050020044880470448004711
:1000D000FEE7FEE7FEE7FEE7FEE7FEE72F13000878
:1000E000B100000830B50B46014600202022012453
:1000F00009E00D46D5409D4205D31D469540491B5C
:100100002546954040191546521E002DF1DC30BDA4
:10011000F0B51FB40646002082B005464024019188
:1001200000901BE0019922460F46304600F020F86F
:10013000049A059B801A994110D31046194622460D
:1001400000F039F8361A8F4101972246012000212C
:10015000009F00F030F838184D4100902046641E92
:100160000028DFDC019B00982946324607B0F0BD2D
:1001700010B5202A04DB0846203AD040002110BDEB
:100180000B46D340D0402024A21A91400843194680
:1001900010BDD2B201E00270401C491EFBD2704774
:1001A0000022F6E710B513460A4604461946FFF743
:1001B000F0FF204610BD10B5202A04DB0146203A8E
:1001C0009140002010BD914020239C1A0346E3403B
:1001D0001943904010BD0000064C0125064E05E075
:1001E000E36807CC2B430C3C98471034B442F7D358
:1001F000FFF762FF4C1B00086C1B000830B501467E
:1002000020314B780022022B04D0042383630A7030
:10021000012030BD03681C680E25AC431C600368D8
:100220001C68640864001C600123056C1C46C06BDC
:10023000AC4044604B700A70002030BD70B50024A3
:10024000014620314A78022A03D004218163012427
:1002500016E0026813680E25AB431360026813684A
:100260005B085B0013600122056C1346AB40C56B55
:100270006B604A7000220A70416B002900D08847E9
:10028000204670BD70B5044600F036F90546601C86
:1002900002D004480078241800F02EF9401BA04238
:1002A000FAD370BD0C000020F0B5002258E0012305
:1002B00093401C460C4052D096082B4DB600751941
:1002C000AF68AC4695072E0F0F25B540AE463D40B2
:1002D0000927FF06B84201D100270FE0234FB8429B
:1002E00001D101270AE0224FB84201D1022705E0DF
:1002F000204FB84201D1032700E00527B740AF42A5
:1003000012D11D4D2E68A6432E606E68A6436E6006
:10031000AE68A643AE60EE68A643EE606546AD6883
:100320007446A5436446A560056856000324B4409E
:10033000A5430560D508AD002D182E6AAC465507BB
:10034000EF0E0F25BD40AE4365462E62C568A5433E
:10035000C56045689D4345608368A3438360521C24
:100360000B46D340A3D1F0BD00000140000400487B
:1003700000080048000C004800040140FCB50023C0
:100380000124A1E027462A469F403A4073D04D6899
:10039000012D05D0022D03D0112D01D0122D16D123
:1003A00085680326AC465D00AE46AE406546B54363
:1003B000AC46CE687546AE4065462E4386604668BC
:1003C0000D79BE43ED06ED0F9D4035434560C6688F
:1003D0005F000325BD40AE46AE4335468E68BE4045
:1003E0002E43C6604E68022E01D0122E14D1DE08B4
:1003F000B60036180196366A5D07B446EE0E0F2534
:10040000B54000966646AE43B4460D69009EB540C1
:1004100066462E43019D2E6206687546AE430D79F1
:10042000AD07AD0FBD40354305604D68ED004AD5C1
:10043000284DAE692643AE61AD699E08ED07ED0F0C
:100440000095254DB6007519AC46AD689E07360F70
:100450000F27B740BD430927FF06B84201D1002747
:1004600010E01E4FB84201D101270BE01C4FB842EB
:1004700002D1022706E026E01A4FB84201D1032735
:1004800000E00527B7402F436546AF60164E35683C
:100490004F689543FF0300D51543356075684F6875
:1004A0009543BF0300D515437560B5684F68954304
:1004B000FF0200D51543B560F5684F689543BF024C
:1004C00000D51543F5605B1C0A681546DA4000D07C
:1004D00058E7FCBD00100240000001400004004845
:1004E00000080048000C004800040140002A01D028
:1004F00081617047816270470148806870470000E1
:100500000C000020024881680278891881607047D9
:100510000C00002010B5064801681022114301604C
:10052000002000F007F800F027F8002010BD0000C0
:100530000020024070B504460D4D7D202978C00092
:10054000FFF7D0FD01460B480068FFF7CBFD00F038
:1005500053FB002809D1042C07D200222146401E5B
:1005600000F03AF800206C6070BD012070BD000002
:100570000C0000200800002008B50848816901220D
:1005800011438161816911400091C26901040A43EC
:10059000C261C0690840009008BD00000010024020
:1005A000002809DBC106C90E012088400349086004
:1005B000BFF34F8FBFF36F8F7047000080E100E003
:1005C000002805DBC106C90E0120884001490860EA
:1005D0007047000000E100E010B501F037FA10BDEF
:1005E000F8B505460068354CC00352D5E0690026D1
:1005F000C00007D4E16920040143E161E1690140E1
:10060000012600912E480168C90510D401688215A1
:1006100011430160FFF770FF074604E0FFF76CFF2E
:10062000C01B642824D826480068C005F6D5206A77
:1006300003273F02384020D06968394081421CD0EE
:10064000206A226AB843012109040A432262226A0D
:100650008A4322622062C0070FD0FFF74DFF00904F
:1006600008E0FFF749FF0099411A1648814201D975
:100670000320F8BD206A8007F3D5206A6968B84373
:1006800008432062002E04D0E16901200007814365
:10069000E1612878C00705D0206BA9688008800038
:1006A000084320632878800605D5206B10218843F5
:1006B000E968084320630020F8BD000000100240F4
:1006C0000070004088130000F8B50F46060059D0AE
:1006D0003A4D2868C007C00FB84209D228684008C0
:1006E0004000384328602868C007C00FB84249D18D
:1006F0003068334C81070CD5400704D5606807216A
:100700000902084360606068F0218843B1680843CB
:1007100060603078C00726D0706801280ED021684C
:1007200002280ED0890700292CDA6168890889001F
:1007300001436160FFF7E0FE00900DE0216889034E
:10074000F1E78901EFE7FFF7D7FE0099411A1D484D
:10075000814201D90320F8BD60680C21084071680E
:1007600089008842EFD12868C007C00FB8420BD972
:10077000286840084000384328602868C007C00F38
:10078000B84201D00120F8BD3078400706D5606836
:10079000072109028843F1680843606000F028F8E7
:1007A0006168094A0906090F515CC8400749086099
:1007B0000020FFF7BFFE0020F8BD0000002002402F
:1007C0000010024088130000341B000808000020BD
:1007D0000448054900684968044A4905490F515CC5
:1007E000C84070470800002000100240441B000869
:1007F00010B514A30FCB88B06C460FC415A30FCB54
:100800000FC4184A51680C200B4603401648042BAD
:1008100016D0082B14D18B021B0F6C46E45CD26AF5
:1008200004AB1207120F9A5CC90305D500231946C1
:10083000FFF76EFC214601E020460C4901F0EEF87E
:1008400008B010BD02030405060708090A0B0C0DC9
:100850000E0F10100102030405060708090A0B0C0D
:100860000D0E0F100010024000127A0000093D002A
:10087000FEB5040070D02078DC4DC0074AD068680F
:100880000007800F012807D068680007800F022842
:1008900009D16868C00306D5286880033AD5606826
:1008A0000028E7D036E06168012914D001208004D7
:1008B000002901D0052914D02A68012109048A439E
:1008C0002A602968814329606068002816D0FFF7F4
:1008D00013FE06460EE0286801210904084328603B
:1008E000F2E7296801432960F5E7FFF705FE801B61
:1008F00064286ED828688003F7D50BE0FFF7FCFD6D
:10090000064604E0FFF7F8FD801B6428F1D828684C
:100910008003F7D420780126800700283CDA686835
:100920000007800F07D068680007800F022809D1F0
:100930006868C00306D42868800716D5E0680128D7
:100940000AD112E0E0680028286816D030432860F9
:10095000FFF7D2FD074605E043E1FFF7CDFDC01BE1
:100960000228C6D828688007F7D52868F821884368
:100970002169C900084328600EE040084000286053
:10098000FFF7BAFD074604E0FFF7B6FDC01B0228DB
:10099000AFD828688007F7D42078000722D5E0690F
:1009A0000028686A0ED030436862FFF7A5FD07464D
:1009B00004E0FFF7A1FDC01B02289AD8686A8007EF
:1009C000F7D50FE0400840006862FFF795FD074645
:1009D00005E09DE0FFF790FDC01B022889D8686AFA
:1009E0008007F7D4207804274007002860DA002029
:1009F0000190E869C00008D4E969B8060143E961DB
:100A0000E969014001200091019079480168C90518
:100A100011D40168821511430160FFF76DFD00904C
:100A200005E0FFF769FD0099401A642870D8704806
:100A30000068C005F5D5A06801280AD0002801D0BB
:100A4000052810D0286A400840002862286AB84368
:100A500001E0286A30432862A068002812D0FFF71E
:100A60004BFD00900AE0286A38432862F1E7FFF75F
:100A700043FD0099411A5F48814249D8286A80079E
:100A8000F5D50DE0FFF738FD009006E0FFF734FDE7
:100A90000099411A574881423AD8286A8007F5D40C
:100AA0000198002804D0E969012000078143E96129
:100AB0002078C00635D5606901280CD0401D686BD0
:100AC00023D038436863686B400840006863FFF7D1
:100AD00013FD064622E0686B38436863686B304359
:100AE0006863FFF709FD064604E0FFF705FD801B7C
:100AF00002285BD8686B8007F7D5686BF8218843BC
:100B0000A169C900084368630BE0B8436863F4E770
:100B10004CE0FFF7F1FC801B022847D8686B800788
:100B2000F7D4206A00285ED069680907890F022976
:100B300042D0012636060228286805D0B043286036
:100B4000FFF7DAFC044633E0B0432860FFF7D4FC3B
:100B5000074604E0FFF7D0FCC01B022826D828680F
:100B60008001F7D4E86AE16A000900010843E862FD
:100B7000616AA06A084369683D22120491430843F0
:100B80006860286830432860FFF7B6FC044604E03C
:100B9000FFF7B2FC001B022808D828688001F7D5AF
:100BA00021E0FFF7A9FC001B022801D90320FEBDAC
:100BB00028688001F5D416E00128F8D06868E96A51
:100BC00001221204636A02409A420AD10907E26ACA
:100BD000090F914205D10F2189040840A16A88427A
:100BE00001D00120FEBD0020FEBD0000001002402B
:100BF0000070004088130000094910B5401E88426B
:100C000001D9012010BD074C60610321081F00F0CD
:100C10001DFF0020A06107202061002010BD000002
:100C2000FFFFFF0000E000E070B5040005D025469E
:100C30002035687F002802D006E0012070BD00202A
:100C40002877204600F014F802206877211D2068DC
:100C500000F06EFB01204034A071A877E877207087
:100C60006070A070E070207160716877002070BDC6
:100C700008B500680549884207D10548C269811551
:100C80000A43C261C0690840009008BD00200040CE
:100C90000010024010B586B0044614216846FFF7E4
:100CA0007FFA0E492068884215D10D484269090132
:100CB0000A434261406908400590102000900220DC
:100CC00001900020029003900420049009206946BE
:100CD000C006FFF753FB06B010BD00000020004027
:100CE00000100240F8B5064604462036307F0D4617
:100CF00001280BD0012008273077002A08D0042AC9
:100D000016D0082A2AD00C2A4DD137E00220F8BD8F
:100D1000206800F049FB20688169394381612068BF
:100D20008169042291438161206881692A6912E006
:100D3000206800F075FB206881690122D20211430E
:100D4000816120688269012189028A438261206869
:100D500081692A6912021143816124E0206800F050
:100D600099FB2068C1693943C1612068C1690422C7
:100D70009143C1612068C1692A6912E0206800F0CE
:100D8000C5FB2068C1690122D2021143C1612068FC
:100D9000C269012189028A43C2612068C1692A6946
:100DA00012021143C16100203077F8BD70B5040014
:100DB00005D025462035687F002802D006E00120B6
:100DC00070BD00202877204600F014F802206877D4
:100DD000211D206800F0ACFA01204034A071A877F2
:100DE000E87720706070A070E070207160716877A3
:100DF000002070BD7047704770470000F8B502686A
:100E00000446D069116896687B4B05461D40202337
:100E1000002D6CD0F707794DFF0FBC460D402F43D6
:100E200079D02546C7078035002F06D0CF0504D5D9
:100E3000012717622A683A432A60820708D5F20719
:100E400006D0276802223A622A6804273A432A60B9
:100E5000420708D5F20706D02668042232622A68C3
:100E6000022632432A6002070AD50A461A4066461D
:100E7000324305D02668082232622E6816432E605F
:100E8000020508D54A0106D501222668D20232623F
:100E90002A681A432A602A68002A30D0800606D5BC
:100EA000880604D5616E002901D02046884728684D
:100EB00021688968490602D42821084225D02046A5
:100EC00000F0F6FB20688168490619D58268402148
:100ED0008A438260206F002812D049494163206F05
:100EE000FFF7ACF900280AD0206F416B06E08506B9
:100EF00011D58D060FD5616E6BE020468847F8BD91
:100F00002046FFF779FFF8BD05E02046FFF774FFA4
:100F100000202860F7E7256E012D55D1C50653D571
:100F2000CD0651D5102616622068816825464906EF
:100F30004035002929DA226F116849680904090C33
:100F4000E1D02F8B8F42DED969839169202917D098
:100F500001683201914301602068816849084900B5
:100F600081602068826840218A438260E3670020B4
:100F7000206620680168B1430160206FFFF73EF9E9
:100F8000288B698B401A81B21AE0298B6A8B891AE7
:100F90006A8B89B2002AB6D00029B4D00268FF2536
:100FA0002135AA430260206882685208520082609C
:100FB000E36700202066606620680268B243026032
:100FC0002046FFF718FF9EE7050605D50D0603D559
:100FD000A16E002991D196E7400694D5480692D596
:100FE0002046146840218C43146083670021816689
:100FF00000F0DCF887E700000F0800002001000483
:101000009D16000810B5040003D0A06F002802D080
:1010100007E0012010BD002174200155204600F09A
:101020003FF82420A0672068016849084900016052
:10103000204600F0CDFB0128ECD0606A002802D0E9
:10104000204600F093FA206841680122D2029143C1
:1010500041602068816808229143816020680168AE
:10106000012211430160204600F0E6FA10BD0000A5
:1010700010B50068084988420DD1084881690122ED
:1010800092039143816109200C21C006FFF70CF9FE
:101090001B20FFF785FA10BD003801400010024008
:1010A00010B586B0044614216846FFF779F8164952
:1010B0002068884226D115488269012189030A43A4
:1010C000826182690A4005924269C9000A4342610D
:1010D0004069084005900C200090022001900020FB
:1010E0000290032003900120049009206946C00665
:1010F000FFF744F9002211461B20FFF76DFA1B2071
:10110000FFF75EFA06B010BD003801400010024043
:1011100030B5C36F202B24D100290BD0002A09D071
:10112000012483682403A34206D10369002B03D161
:10113000CB0701D0012030BD034660331C7D012C5C
:101140000FD001241C750023036603685C68240229
:1011500004D51C680125AD062C431C6000F0C6FBBD
:1011600030BD022030BD000010B50E49006809688E
:10117000884216D10C480B4BC188027884335A54EC
:10118000491C8BB20021C380662B00D1C180232A69
:1011900002D1C18001214170012203490148FFF7BA
:1011A000B7FF10BD60000020000000207047FEE780
:1011B000F0B587B014216846FEF7F2FF1D4842697A
:1011C000012149040A43426142690A400592426989
:1011D00049000A4342614069174D08400926F60656
:1011E0000590002229463046FFF780F9134F002270
:1011F00002213846FFF77AF9032000240090019479
:10120000694602943046FFF7B9F80095012502942B
:101210006946304601950394FFF7B0F8022000902C
:1012200002946946019503943846FFF7A7F807B082
:10123000F0BD000000100240E0660000000400481D
:1012400010B588B01C216846FEF7AAFF0E490F486A
:10125000002412C0046084600D49046141600838B4
:10126000FFF7E2FC0948FFF7A1FD60200090019420
:1012700002940022694604940448FFF733FD0348B2
:10128000FFF708FD08B010BD002000401800002046
:10129000FFFF000010B50A48084901604B21C90151
:1012A000416000218160C16001618161C1610C22E6
:1012B000016242614162FFF7A5FE10BD00380140A6
:1012C0006000002070477047704710B5FFF71AF9AB
:1012D00010BD70B594B030216846FEF761FF002460
:1012E0000E94139410200994022504900D940F94E9
:1012F0000520129401260095C0040C9410940396C6
:101300000A90119408950B946846FFF7B1FA0720EC
:101310000C900E9401210D950F940CA8FFF7D4F9B1
:1013200010A810961294FFF75BF914B070BD7047C7
:1013300070B50268174B184E984201D0B04203D1E5
:101340007024A2434C682243144C154D984208D097
:10135000B04206D0134EB04203D0A04201D0A84202
:1013600004D103263602B243CE6832438026B2430C
:101370004E69324302608A68C2620A688262984299
:1013800003D0A04201D0A84201D109690163012123
:10139000416170BD002C0140000400400044014048
:1013A0000048014000200040F0B5026A5208520097
:1013B0000262056A436882697024A24392080C683D
:1013C00092001443022295438A68134E2A43114D1A
:1013D000A84204D0B04202D0104FB84206D108272C
:1013E000BA43CF681743042297433A46A84204D031
:1013F000B04202D0094DA84206D103252D02AB43CD
:101400004D691D438B692B43436084614968416387
:101410000262F0BD002C0140004401400048014040
:1014200070B5026A10239A430262046A43688269B3
:1014300073252D02AA430D682D02154320229443E3
:101440008A6812012243104CA04208D11446CA688F
:101450008026B443120122434024A24305E00B4CF2
:10146000A04202D00A4CA04208D10324A402A34304
:101470004C69A4001C438B699B0023434360856136
:1014800049688163026270BD002C01400044014044
:101490000048014070B5026AFF2301339A4302629B
:1014A000046A4368C2697025AA4392080D689200D5
:1014B00015430122520294438A6812022243104CBF
:1014C000A04207D1C414A243CC68240222430615CB
:1014D000B24305E00B4CA04202D00B4CA04208D115
:1014E00003242403A3434C6924011C438B691B017F
:1014F00023434360C5614968C163026270BD000057
:10150000002C0140004401400048014030B5026A0F
:1015100001231B039A430262056A4268C36973246C
:101520002402A3430C6824021C4301235B039D4354
:101530008B681B032B430A4DA84205D0094DA842D6
:1015400002D0094DA84205D10125AD03AA434D693A
:10155000AD012A434260C46149680164036230BD41
:10156000002C0140004401400048014010B5818C2E
:10157000C90707D001684A6801235B049A43836A5C
:101580001A434A60818C890707D501684A6801239C
:101590001B049A43C36A1A434A60818C490707D5E2
:1015A00001684A6801239B049A43036B1A434A600B
:1015B000818C090707D501684A680123DB039A4338
:1015C000436B1A434A60818CC90607D5026891684B
:1015D00001231B039943836B19439160818C890616
:1015E00007D501688A6801235B039A43C36B1A43DA
:1015F0008A60818C490612D503685A680121090561
:10160000046C8A4322435A60026C8A4207D1026802
:10161000516803235B059943436C19435160818CE6
:10162000090607D501684A680123DB04806C9A43E8
:1016300002434A6010BD0000F8B504460026803021
:101640000660FEF759FF054620680068124F000744
:1016500009D501212B46002249052046009700F0BC
:1016600085F900280DD12068006840070BD50121BD
:101670002B46002289052046009700F077F90028C4
:1016800001D00320F8BD2020A067E0672666603403
:1016900026750020F8BD0000FFFFFF0110B5406A6D
:1016A0000022014640314A834A82FFF7A5FB10BD64
:1016B00001680A68FF2321339A430A6001688A6837
:1016C000520852008A60016E012904D101680A683B
:1016D00010239A430A602021C167002101664166F8
:1016E000704770B504464030828BE36F2168222B2F
:1016F00004D0886908221043886170BD898C636DAD
:1017000011401980616D891C6165418B491E4183BF
:10171000418B0029F1D121680A68FF2321339A43C4
:101720000A6021688A68520852008A602021E167B5
:1017300000256566216E012904D02046FFF714FDBF
:10174000256670BD21680A6810239A430A60018BE0
:101750002046FFF750FBF3E770B504464030828B1C
:10176000E36F2168222B04D0886908221043886126
:1017700070BD898C1140626D1170616D491C61658D
:10178000418B491E4183418B0029F1D121680A68B0
:10179000FF2321339A430A6021688A685208520065
:1017A0008A602021E16700256566216E012904D049
:1017B0002046FFF7D9FC256670BD21680A68102312
:1017C0009A430A60018B2046FFF715FBF3E7000000
:1017D00070B5044680682169E269084361690025A3
:1017E0001143084321680A683C4B1A4002430A60CF
:1017F00021684868032212039043E268104348605E
:10180000A169206A084321688A680B231B029A4356
:1018100002438A603248006B8007800F16D001288F
:1018200018D0022818D0032812D010210120E36913
:10183000C0032C4A2C4E83422BD100290ED0022902
:101840000FD004290FD008293FD110E00021EDE787
:101850000221EBE70421E9E70821E7E7FEF7B8FFFB
:1018600003E0104603E0FEF7C3FF002831D06168B3
:1018700040004A088018FEF735FC80B20146103956
:10188000B14222D81849491C01400007400F0843C3
:101890001DE0002906D0022907D0042907D0082915
:1018A00013D108E0FEF794FF03E0104603E0FEF7D3
:1018B0009FFF00280DD061684A081018FEF712FC3F
:1018C00080B201461039B14201D9012501E02168F9
:1018D000C86000206066A066284670BDF369FFFFFF
:1018E0000010024000127A00EFFF000030B54165A1
:1018F000014640310A834A830022426601238568FB
:101900001B03FF249D4204D10569002D23D1144CF3
:1019100021E0002D1BD08A8380210A502221C1673B
:1019200001688C6801252C438C608168994202D142
:101930000169002911D00B49416674210A540068DD
:101940000168FF22213211430160002030BD05698A
:10195000002D00D07F248C83DEE70349ECE70000F4
:10196000FF01000059170008E3160008FFB581B019
:1019700005460F46044660350A9E39E0701C37D094
:10198000FEF7BAFD0499401AB04222D8002E20D0AA
:101990002068016849072BD5C069C043000527D4DA
:1019A00001202168C002086220680168FF22A1327C
:1019B00091430160206881684908490081602020C6
:1019C000A067E0678034206000202875032005B000
:1019D000F0BD20680168FF22A132914301602068B8
:1019E00081684908490081602020A067E067EBE733
:1019F0002068C1693846884305D000210398814298
:101A0000BCD00020E3E70121F8E7000010B5024850
:101A1000FFF7F4F910BD000060000020F8B5040CD9
:101A20008BB2264682B25E430D0C1046370C5843EB
:101A3000360480190021794116466E43370C36046E
:101A40008019794126466E438919F8BD8307FF2224
:101A5000DB0E9A408907090E9940002808DB8308AD
:101A600009489B001B18186890430843186070478A
:101A70000007000F0838830804489B001B18D8692A
:101A800090430843D861704700E400E000ED00E0B7
:101A900002E008C8121F08C1002AFAD17047704737
:101AA000002001E001C1121F002AFBD17047000095
:101AB000FEF730FDFFF70DFCFFF77AFBFFF7EAFBBF
:101AC000FFF7BEFB1948FFF7D3FA7D20C000FEF7F1
:101AD000D9FB1648FFF7E4FA6420FEF7D3FBFFF7C3
:101AE000D9FB002211461B20FEF776FD1B20FEF7D6
:101AF00067FD01220E490D48FFF70AFBFF2601246E
:101B0000F53664030925ED063046FEF7BBFB0122DE
:101B100021462846FEF7EAFC3046FEF7B3FB0022DA
:101B200021462846FEF7E2FCEEE7000060000020B8
:101B3000000000200000000000000000010203047B
:101B40000607080900000000010203046C1B0008DE
:101B50000000002018000000901A0008841B0008F4
:101B60001800002030050000A01A000800000D0A2F
:101B70006500000000127A0001000000040000006F
:041B80000000000061
:04000005080000B13E
:00000001FF
